:106fa0008058900000c2b30080cf5000050032002e
:106fb000304080008058900000c3b30080cf500064
:106fc00012003a00304080000009900090099000c3
:106fd000304080007000900001002000800f5100c0
:106fe000818f59000f013900324080006000b800e5
:106ff0000009980011099800314080000158900064
:107000000040e800805898000601370030408000ba
:10701000c00090002e009000808f500009003e00bc
:1070200030408000000990009009900030408000be
:10703000e000900050009000800f5100818f5900b7
:10704000f800390031408000214090000060a0002d
:10705000a040980031408000015890000040e800b6
:1070600080589800ef0037001e00900090007800d4
:1070700000c023008080600000c02000808f50008e
:10708000070032001e0090009000780000c023002e
:107090008080600000c02200808f500036003a00df
:1070a0009e009000f03f2000110060002007980033
:1070b000344080003040800000099000900990002a
:1070c0002e00900001002000020040008380480054
:1070d000000a9800110a9800314080000000eb007f
:1070e0008010980030408000304090006240600086
:1070f0000004e00005003200314080003140900083
:107100000010a100b040980004003700314080001a
:10711000314090000010a000b04098003040800046
:10712000c00090002e009000808f500009003e00ab
:1071300030408000000990009009900030408000ad
:10714000e000900050009000800f5100818f5900a6
:10715000b400390031408000214090000060a00060
:10716000a040980031408000015890000040e800a5
:1071700080589800ab0037001e0090009000780007
:1071800000c023008080600000802200808f5000bb
:1071900065003a0031408000314090000020a0009e
:1071a000b040980031408000011090000000e800dd
:1071b000801098003040800050589000634060007c
:1071c0000080fb00400798004e009000e10f500047
:1071d0004c0032004e009000e10f500004003c00d3
:1071e0004e0090000000e000190032008d003700d2
:1071f0004e009000e20f5000040032004e0090005c
:10720000e30f50002200320086003700304080003b
:107210008010900000712200808f500081003600a5
:107220003140800070c1b300e058980032408000c7
:10723000304080000058900080407800f0c0b300db
:1072400000c06000f040b30000599800750037009e
:107250003040800000109000f40f500071003600a4
:107260003140800070c1b300e05898003240800087
:10727000304080000058900080407800f0c0b3009b
:1072800000c06000f040b30000599800650037006e
:1072900030408000405890000004e00010003500ad
:1072a0003040800000109000f40f50005d00360068
:1072b0003140800070c1b300e05898003240800037
:1072c000304080000058900080407800f0c0b3004b
:1072d00000c06000f040b300005998005100370032
:1072e00031408000214090000060a000a040980044
:1072f00031408000015890000040e800805898001c
:107300004800370031408000214090000060a0001c
:10731000a040980031408000015890000040e800f3
:10732000805898003f0037001e00900090007800c1
:1073300000c023008080600000802300808f500008
:1073400010003a0031408000214090000030a00041
:10735000a04098003140800010c1b300e058980070
:10736000324080003040800000589000804078001b
:10737000f0c0b30000c06000f040b30000599800b6
:1073800028003700324080002240900067406000b3
:107390000040e80067406000a2409000e7416000c4
:1073a00080cfb30080c0600083c07000214198008e
:1073b0003040800020409000674060000080fb006b
:1073c000e20f50001700340031408000214090004f
:1073d0000030a000a0409800314080002140900083
:1073e0000040a000a04098003140800030c1b300b0
:1073f000e0589800324080003040800000589000f3
:1074000080407800f0c0b30000c06000f040b300de
:1074100000599800f00f2000702488002000200000
:107420005024880022f807008cc4bf00644060002c
:107430000004e000400032008ac4bf0064406000e5
:107440000004e0003c00320040002000502488008e
:10745000a0488000100f78001d0037001e00780043
:10746000e0089000003020008080600000302000a4
:10747000808f5000070032001e007800e008900066
:10748000003020008080600000102000808f5000bd
:1074900009003a001e007800300090000000e00073
:1074a000050032001e007800300090008000e900e6
:1074b0001e007800310098001e007800b040900057
:1074c0000120a100314098001e007800100f7800c4
:1074d0001e00e000e1ff3a008180200011407800aa
:1074e0000000a100804878008180200011407800d1
:1074f0000010a100804878008180200011407800b1
:107500000020a10080487800818020001140780090
:107510000030a10080487800828020006000b80020
:107520001001980021019800818020000040eb00ac
:10753000e0409800def707008cc4bf0062406000a6
:107540000004e0005c0032008ac4bf0062406000ba
:107550000004e00058003200200020005024880081
:107560003240800022409000674060000040e80008
:1075700067406000a2409000e741600080cfb30008
:1075800080c0600083c070002141980030408000be
:1075900020409000674060000080fb00e20f500038
:1075a0004500340031408000214090000030a000b0
:1075b000a0409800e14820009140780000c8b30046
:1075c00000c060000004e000030032003140800091
:1075d00000c2b300e05898008ec4bf000042b20061
:1075e0000004e000030032003140800010c2b3000c
:1075f000e05898008ec4bf00704060000004e000b6
:10760000030032003140800020c2b300e0589800ef
:107610008ec4bf00684060000004e0000300320038
:107620003140800030c2b300e05898008ec4bf00e3
:10763000644060000004e00003003200314080003c
:1076400040c2b300e05898008ec4bf0062406000a2
:107650000004e000030032003140800050c2b3005b
:10766000e05898008ec4bf00614060000004e00054
:10767000030032003140800060c2b300e05898003f
:10768000f00f2000702488003140800021409000dd
:107690000040a000a04098003240800030408000b0
:1076a0000058900080407800f0c0b30000c0600037
:1076b000f040b300005998000080fa003400f9004f
:1076c0004f03be004f02be004f01be004f00be0080
:1076d0003600f900004006000800fa002047980034
:1076e0000040eb0010479800030037001e40900058
:1076f0000040e800104798001e4090000004e000a1
:107700000a003a001e4090000080fb007400b9009f
:10771000ea004000a08f20000080400090407800e8
:107720002e40900080cf5000f0ff3a001e409000a5
:10773000e14f500003003a00300520003007980068
:107740003e0037002e409000a5ee0700004f780065
:1077500000c3b3009e4f1000030032009e80fb0068
:1077600031079800350037001e4090000080fb0074
:107770007400b900ec004000a08f200000804000a1
:10778000104078008080fb00000f200080806000a7
:107790002107980000032000ae009000808f500069
:1077a0001b00320000032000ae009000808f5000cc
:1077b00008003c002e009000f00f50000e00320038
:1077c00000022000ae009000808f50000d003200bb
:1077d0001800370000042000ae009000808f500099
:1077e0001100320000062000ae009000808f500093
:1077f0000a0032000f003700100520003007980003
:107800000e00370021052000310798000b003700db
:10781000300520003007980008003700410520009f
:107820003107980005003700500520003007980008
:107830000200370001052000310798003e0090004b
:107840000080fa00000006000600fa0020479800b9
:107850002e4090000004e000030032002e40900013
:107860000004e00003003d003005200020079800e0
:107870004f0037000040eb00004f78000100370058
:107880001e4fe8001e04e00009003a001e80fb00c5
:107890007400b900ea004000a08f20000080400082
:1078a000904078002e40900080cf5000f4ff3a00c6
:1078b00010c0b3009e4f100003003a0030052000b6
:1078c000200798003a0037001e80fb007400b900c2
:1078d000ec004000a08f20000080400010407800a5
:1078e0008080fb00000f2000008060000000e000ae
:1078f0002d0032001e80fb007400b900ec00400037
:10790000a08f200000804000104078008080fb00a5
:10791000000f200000806000f00f500022003200b5
:107920009e81fb001e80fb007400b900e80040004f
:10793000a08f2000008040001040780000417800b7
:10794000e240b3007418b900800078002090200055
:1079500000804000024878001e80fb007400b900df
:107960008000780020902000808040001100780086
:107970000010a000800878001e80fb007400b90091
:1079800080007800609020008080400000c6b30036
:10799000904098001e407800e70707000000eb00c9
:1079a0002007980002003700b0052000200798004b
:1079b0002e0090000080fa00000006001200fa007d
:1079c000881f78000040eb00004f7800b4043700b7
:1079d0001e80fb007400b900ea004000a08f200068
:1079e00000804000104078000004e00007003a00ea
:1079f0001e80fb007400b9008000780060902000b9
:107a0000808040000040eb00804878001e80fb0032
:107a10007400b900ec004000a08f200000804000fe
:107a2000104078008080fb00000f20008080600004
:107a3000010f9800000220008e089000808f5000f7
:107a400052003200000220008e089000808f50000b
:107a500007003c000e0890000000e0008f04320098
:107a60008e089000f08f50000a0032008b0437001f
:107a7000000320008e089000808f5000ea01320041
:107a8000000420008e089000808f5000d203320046
:107a9000820437001e80fb007400b900ec00400037
:107aa000a08f200000804000104078000080fb0084
:107ab0006f006000700798007e0090000000e000fa
:107ac00004003200fe009000e18f50001d003200e3
:107ad000720437001e80fb007400b900ea00400009
:107ae000a08f20000080400010407800bced07000f
:107af0008040780000c3b30080cf500067043a0094
:107b00009e81fb001e80fb007400b900ec00400069
:107b1000a08f200000804000104078000040e80066
:107b2000004178007418b90080007800609020004f
:107b300000804000024878002049800030498800d9
:107b4000560437009e81fb001e80fb007400b900c4
:107b5000ec004000a08f2000008040001040780022
:107b60008040780000cfb30000c06000704040004b
:107b7000004178007418b9008000780060902000ff
:107b80000080400002487800440437001e80fb005b
:107b90007400b900ec004000a08f2000008040007d
:107ba000104078000080fb006f00600060079800c4
:107bb0006e009000e20f5000b3003200ee00900023
:107bc000e28f500007003c006e0090000000e000d3
:107bd0000b003200ee009000e18f50007300320085
:107be0002e0437006e009000e30f5000b500320005
:107bf000ee009000e48f50000101320027043700ae
:107c000094c4bf000042b2000004e00023043a0024
:107c1000304980000000e00055003200304980000b
:107c2000100090000000e0001c0432001e84fb00e5
:107c3000304980001000900040eb07000001780000
:107c40007440b90080007800e08f20000080400080
:107c5000020878007440b900e4004000a08f2000c2
:107c600000804000100078000000e0000f003a00a3
:107c70001e80fb007400b900800078004090200056
:107c80008080400050c0b300904098001e80fb00f0
:107c90007400b9008000780060902000808040006f
:107ca00000c6b30080487800fc0337001e80fb004c
:107cb0007400b900e4004000a08f20000080400064
:107cc0001001780030498000900190003049800018
:107cd000004890000082fb001e80fb007400b90089
:107ce000ea004000a08f2000008040001040780093
:107cf00017c0b3000203780083027800032022003b
:107d000062c0b30011c8b300d0ec07000004e0006b
:107d10000f003a009e81fb001e80fb007400b9003a
:107d2000ec004000a08f2000008040001040780050
:107d30000040e800004178007418b9008000780025
:107d4000609020000080400002487800d303370094
:107d50001e80fb007400b900e4004000a08f2000ea
:107d6000008040001000780046eb0700cb0337008e
:107d70001e80fb007400b900800078004090200055
:107d80008080400060c5b300904098001e80fb00da
:107d90007400b9008000780060902000808040006e
:107da00000c6b30080487800bc0337001e80fb008b
:107db0007400b900ea004000a08f2000008040005d
:107dc000104278000e80e8006601470080017800cc
:107dd0008040eb0004407800f7f307000000e0006b
:107de000ae0332006e4090000004e0000f0032004d
:107df0001e80fb006e4190007400b9008000780086
:107e00004090200000804000124098001e80fb003f
:107e10007400b900800078006090200080804000ed
:107e200000c6b30080487800080037001e80fb00c1
:107e30007400b900ea004000a08f200000804000dc
:107e4000104078008040eb0059ec07009e81fb0059
:107e50001e80fb007400b900ec004000a08f2000e1
:107e600000804000104078000040e80000417800a9
:107e70007418b900800078006090200000804000f5
:107e800002487800850337009e81fb001e80fb00be
:107e90007400b900ec004000a08f2000008040007a
:107ea000104078000040e800004178007418b900e4
:107eb0008000780060902000008040000248780038
:107ec000760337001e84fb00304980000049900093
:107ed00030498000104890008082fb0030498000cb
:107ee000100290001e80fb007400b900e400400006
:107ef000a08f2000008040001000780082417800b0
:107f00000501780084007800b906070000017800b8
:107f10007440b9008000780000902000008040008c
:107f2000020878001e80fb007400b900e6004000e3
:107f3000a08f200000804000100078000000e000ca
:107f400020003200c07c29004d1707001e80fb0076
:107f50007400b900ea004000a08f200000804000bb
:107f6000104090000080fb00951707001e80fb006a
:107f70007400b900ea004000a08f2000008040009b
:107f800010407800320607001e80fb007400b90024
:107f900080007800409020008080400030c0b30016
:107fa000904098001e80fb007400b90080007800ab
:107fb000609020008080400000c6b30080487800b8
:107fc000360337009e81fb001e80fb007400b90061
:107fd000ec004000a08f200000804000104078009e
:107fe0000040e800004178007418b9008000780073
:107ff000609020000080400002487800270337008e
:10800000208d2000100278001e80fb007400b90053
:10801000ea004000a08f200000804000104078005f
:108020006011b80004000100208d20009001900034
:108030001e80fb007400b900ea004000a08f200001
:1080400000804000104078006022b8000001eb0082
:10805000d1122000030001000000e00009003200fe
:108060001e80fb007400b900800078002090200082
:1080700080804000110078000040a0008008780057
:108080002c00370030498000004890000081fb0040
:108090001e80fb007400b900ee004000a08f20009d
:1080a00000804000104078000080fb000000e900e4
:1080b000800f51001f003a001e80fb007400b900c1
:1080c000e8004000a08f20000080400010007800f1
:1080d0004400de00614060000004e00015003a004a
:1080e0001e80fb007400b900ea004000a08f200051
:1080f0000080400010407800d50507001e80fb007e
:108100007400b9008000780040902000808040001a
:1081100030c0b300904098001e80fb007400b9008e
:1081200080007800609020008080400000c6b3008e
:10813000804878001e80fb007400b900e400400015
:10814000a08f200000804000100078004dea07005a
:1081500030498000100078003049880030498000a4
:108160000000e000080032001e80fb007400b9002f
:1081700080007800609020008080400000c2b30042
:1081800080487800c50237001e80fb007400b900eb
:10819000e8004000a08f2000008040001000780020
:1081a0004400de00614060000004e00016003a0078
:1081b0001e80fb007400b900ea004000a08f200080
:1081c0000080400010407800a10507001e80fb00e1
:1081d0007400b9008000780040902000808040004a
:1081e00030c0b300904098001e80fb007400b900be
:1081f00080007800609020008080400000c6b300be
:1082000080487800a50237001e80fb007400b9008a
:1082100080007800609020008080400000c3b300a0
:10822000804878009d0237001e80fb007400b90072
:10823000ec004000a08f200000804000104078003b
:108240000080fb006f006000500798005e00900007
:10825000e30f5000d2003200de009000e38f5000a8
:1082600007003c005e009000e10f50000e0032005d
:10827000de009000e18f500066003c00870237006e
:108280005e009000e50f500065013200de009000b6
:10829000e58f5000d60035005e009000e60f5000dc
:1082a000b90132007d0237001e80fb007400b90066
:1082b000f0004000a08f200000804000104090009f
:1082c0000082fb00050020001e80fb007400b90046
:1082d0008080e800a08f200000804000100178001e
:1082e0001e80fb007400b900f2004000a08f200047
:1082f00000804000904178001e80fb007400b900af
:10830000ea004000a08f200000804000104078006c
:1083100083407800ffeb0700604798006e409000b4
:108320000004e0002c0032006e409000f14f50003d
:108330001a003a001e80fb007400b900ea004000f9
:10834000a08f200000804000104078008040eb00ab
:1083500017eb07001e80fb007400b9008000780056
:10836000609020008080400000c6b30090409800dc
:108370001e80fb007400b90080007800209020006f
:1083800080804000110078000010a0008008780074
:108390001e40780068050700400237001e80fb0081
:1083a0006e4190007400b900800078004090200079
:1083b00000804000124098001e80fb007400b9004d
:1083c00080007800609020008080400000c6b300ec
:1083d00080487800310237009e81fb001e80fb0040
:1083e0007400b900ec004000a08f20000080400025
:1083f000104078000040e800004178007418b9008f
:1084000080007800609020000080400002487800e2
:10841000220237001e80fb007400b900f200400009
:10842000a08f200000804000904278001e80fb005a
:108430007400b900ea004000a08f200000804000d6
:10844000104278000e80e800660147008001780045
:10845000854078000440780057f207000000e000f3
:108460000e0232006e4090000004e0002c0032004a
:108470006e409000f14f50001a003a001e80fb0041
:108480007400b900ea004000a08f20000080400086
:10849000104078008040eb00c5ea07001e80fb001a
:1084a0007400b90080007800609020008080400057
:1084b00000c6b300904098001e80fb007400b90015
:1084c000800078002090200080804000110078001b
:1084d0000010a000800878001e40780016050700f4
:1084e000ee0137001e80fb006e4190007400b90061
:1084f00080007800409020000080400012409800ea
:108500001e80fb007400b90080007800609020009d
:108510008080400000c6b30080487800df0137004b
:108520001e80fb007400b900ea004000a08f20000c
:1085300000804000104078008040eb009cea07007b
:108540001e81fb001e009000ae009000804178006c
:108550007410b90080007800a090200000804000d6
:10856000034878009e81fb001e80fb007400b90068
:10857000ec004000a08f20000080400010407800f8
:108580000040e800004178007418b90080007800cd
:10859000609020000080400002487800bf01370052
:1085a0001e80fb007400b9008000780060902000fd
:1085b0008080400000c3b30080487800208d2000f8
:1085c000900190001e80fb007400b900ea0040009a
:1085d000a08f200000804000104078006022b8008a
:1085e0000001eb000113200003000100ab01370084
:1085f0001e80fb007400b900f2004000a08f200034
:1086000000804000104078000004e00029003a009b
:108610001e80fb007400b9008080e800a08f20005d
:1086200000804000100178001e80fb007400b9003b
:10863000f0004000a08f200000804000104090001b
:108640008081fb001e80fb007400b900ee0040003a
:10865000a08f200000804000104090000082fb00ae
:108660001e80fb007400b90080007800a08f2000fd
:1086700000804000100478001e80fb007400b900e8
:10868000ea004000a08f20000080400010407800e9
:108690008043eb00020378008302780088017800b1
:1086a00092c0b30011c2b30068ea070060479800a7
:1086b0001d0037001e80fb007400b900f000400070
:1086c000a08f200000804000104090000082fb003e
:1086d000050020001e80fb007400b9008080e800c7
:1086e000a08f200000804000100178001e80fb0059
:1086f0007400b900f2004000a08f2000008040000c
:10870000904178001e80fb007400b900ea00400030
:10871000a08f200000804000104078008340780047
:1087200018f20700604798006e4090000004e000d7
:108730002c0032006e409000f14f50001a003a00b9
:108740001e80fb007400b900ea004000a08f2000ea
:1087500000804000104078008040eb0014ea0700e1
:108760001e80fb007400b90080007800609020003b
:108770008080400000c6b300904098001e80fb003f
:108780007400b900800078002090200080804000b4
:10879000110078000010a000800878001e407800ca
:1087a000650407003d0137001e80fb006e4190000c
:1087b0007400b900800078004090200000804000e4
:1087c000124098001e80fb007400b9008000780001
:1087d000609020008080400000c6b3008048780090
:1087e0002e0137009e81fb001e80fb007400b90043
:1087f000ec004000a08f2000008040001040780076
:108800000040e800004178007418b900800078004a
:108810006090200000804000024878001f0137006f
:108820001e80fb007400b900f2004000a08f200001
:1088300000804000904278001e80fb007400b90068
:10884000ea004000a08f2000008040001042780025
:108850000e80e800660147008001780085407800be
:108860000440780054f107000000e0000b013200e2
:108870006e4090000004e0002c0032006e4090003a
:10888000f14f50001a003a001e80fb007400b9003e
:10889000ea004000a08f20000080400010407800d7
:1088a0008040eb00c2e907001e80fb007400b900a5
:1088b00080007800609020008080400000c6b300f7
:1088c000904098001e80fb007400b9008000780082
:1088d0002090200080804000110078000010a0004f
:1088e000800878001e40780013040700eb00370072
:1088f0001e80fb006e4190007400b900800078007b
:108900004090200000804000124098001e80fb0034
:108910007400b900800078006090200080804000e2
:1089200000c6b30080487800dc0037001e80fb00e2
:108930007400b900ea004000a08f200000804000d1
:10894000104078008040eb0099e907009e81fb0011
:108950001e80fb007400b900ec004000a08f2000d6
:1089600000804000104078000040e800004178009e
:108970007418b900800078006090200000804000ea
:1089800002487800c50037001e80fb007400b90063
:1089900080007800609020008080400000c3b30019
:1089a00080487800208d2000900190001e80fb0000
:1089b0007400b900ea004000a08f20000080400051
:1089c000104078006022b8000001eb001113200075
:1089d00003000100b10037001e80fb007400b900e5
:1089e000ec004000a08f2000008040001040780084
:1089f0000080fb006f00600040079800ce009000f0
:108a0000e18f50005b0032004e009000e20f5000fa
:108a1000a0003200ce0090000100e0000100320012
:108a20009e0037001e80fb007400b900ee0040007d
:108a3000a08f200000804000104090000081fb00cb
:108a40001e80fb007400b900ea004000a08f2000e7
:108a500000804000104078008043eb000003eb00f2
:108a60008002eb00020278008001eb0000c1eb0005
:108a700011c2b30075e90700604798006e4090008e
:108a80000004e0002c0032006e409000f14f5000d6
:108a90001a003a001e80fb007400b900ea00400092
:108aa000a08f200000804000104078008040eb0044
:108ab0003fe907001e80fb007400b90080007800c9
:108ac000609020008080400000c6b3009040980075
:108ad0001e80fb007400b900800078002090200008
:108ae00080804000110078000010a000800878000d
:108af0001e40780090030700680037001e80fb00ce
:108b00006e4190007400b900800078004090200011
:108b100000804000124098001e80fb007400b900e5
:108b200080007800609020008080400000c6b30084
:108b300080487800590037009e81fb001e80fb00b2
:108b40007400b900ec004000a08f200000804000bd
:108b5000104078000040e800004178007418b90027
:108b6000800078006090200000804000024878007b
:108b70004a0037001e80fb007400b900ea00400084
:108b8000a08f200000804000104278000e80e80096
:108b900066014700800178008040eb0004407800c7
:108ba00085f007000000e0003c0032006e409000bd
:108bb0000004e0002c0032006e409000f14f5000a5
:108bc0001a003a001e80fb007400b900ea00400061
:108bd000a08f200000804000104078008040eb0013
:108be000f3e807001e80fb007400b90080007800e5
:108bf000609020008080400000c6b3009040980044
:108c00001e80fb007400b9008000780020902000d6
:108c100080804000110078000010a00080087800db
:108c20001e407800440307001c0037001e80fb0034
:108c30006e4190007400b9008000780040902000e0
:108c400000804000124098001e80fb007400b900b4
:108c500080007800609020008080400000c6b30053
:108c6000804878000d0037001e80fb007400b900ba
:108c70008000780020902000808040001100780063
:108c80000010a100800878001e4078002a03070029
:108c9000020037001e407800270307001e4fe8003f
:108ca0001e04e0004afb32004f0478000080fa0006
:108cb000000006000e00fa00204798003147980097
:108cc00042479800330798004407980055079800da
:108cd0000040eb00004f7800010037001e4fe80015
:108ce0001e04e00009003a001e80fb007400b90079
:108cf000ea004000a08f20000080400090407800f3
:108d00002e40900080cf5000f4ff3a0010c0b30016
:108d10009e4f100003003a003105200061079800c3
:108d20007f00370020498000304988000300370069
:108d300030498000100078003049880030498000b8
:108d40000000e000050032003049800080489000bb
:108d50004e40900080cf5000f5ff3a001e80fb008f
:108d60007400b900ec004000a08f2000008040009b
:108d70009040780000c3b30080cf50000d00320057
:108d80001e80fb007400b900ec004000a08f2000a2
:108d900000804000104078000080fb006f00600001
:108da0000000e0000300320040052000600798004a
:108db0005b0037001e80fb007400b9008000780063
:108dc000a0902000808040000040eb0080487800a8
:108dd0001e80fb007400b9008000780040902000e5
:108de000808040000040eb00904098001e80fb0017
:108df0007400b90080007800c08f2000008040001f
:108e0000de009000010878009e80fb003049800061
:108e1000604190007408b90080007800c090200084
:108e200000804000024878009e80fb004e009000c9
:108e3000004178007408b90080007800a0902000fc
:108e400000804000124098001e80fb007400b900b2
:108e500080007800a08f200000804000be009000bd
:108e6000010878001e80fb007400b90080007800c3
:108e70008090200000804000ce409000114098007b
:108e80003e4090000004e00011003a009e80fb008c
:108e900030498000704190007408b900800078006b
:108ea000c090200000804000024878001e81fb0036
:108eb000be00900000202000808170007410b90076
:108ec00080007800a08f2000008040000308780018
:108ed0003e4090000004e00008003a001e80fb00c5
:108ee0007400b9008000780060902000808040000d
:108ef00040c3b30080487800070037001e80fb00a5
:108f00007400b900800078006090200080804000ec
:108f100010c3b300804878000000eb0060079800a1
:108f20006e0090000080fa00000006000a00fa00bf
:108f30002047980021079800320798000040eb0076
:108f4000004f7800010037001e4fe8001e04e000cb
:108f500009003a001e80fb007400b900ea004000de
:108f6000a08f200000804000904078002e409000ac
:108f700080cf5000f4ff3a0010c0b3009e4f1000a5
:108f8000080032001e80fb007400b900ec004000b5
:108f9000a08f200000804000104078000004e00016
:108fa00009003a00ae00900030c5b3008048780058
:108fb000be0090000040eb008048780010002000c8
:108fc000400798001e0037001e80fb007400b900a7
:108fd000f0004000a08f200000804000904078000a
:108fe0003e009000014878001e80fb007400b9002c
:108ff000ea004000a08f20000080400090409000d8
:109000002e009000014878001e80fb007400b9001b
:10901000ec004000a08f20000080400090407800cd
:1090200000c3b30080cf500003003a0010002000be
:1090300040079800020037000000eb00400798004e
:109040004e0090000080fa00000006001000fa00b8
:10905000204798002107980032079800440798009d
:10906000550798002e009000e90f500046003e0082
:10907000110020002e0090008008dd00710798008c
:10908000e0332000fe009000008060000000e0005f
:109090003a003a0000082000fe00900000806000c6
:1090a0000000e0000a003a00fe00900061806000cd
:1090b0000000e00001003a00330037006ae90700d1
:1090c0003efa0700100020006007980030003700cb
:1090d0000040eb00004f7800010037001e4fe80011
:1090e0001e04e00009003a001e80fb007400b90075
:1090f000ea004000a08f20000080400090407800ef
:109100002e40900080cf5000f4ff3a001e04e00093
:1091100017003a001e80fb007400b9008000780040
:1091200040902000808040000040eb0080487800a4
:109130001e80fb007400b900800078006090200061
:10914000808040000040eb0080487800208d2000a7
:10915000900190006022b8000001eb007100200037
:109160002e409000030001001e407800b801070067
:109170001100200061079800050037001000200052
:1091800060079800020037008000eb00610798003c
:109190006e0090000080fa00000006001800fa003f
:1091a00000579800120f9800230f98000000eb0062
:1091b000700798000000eb00600798000000eb00cb
:1091c000500798000000eb00400798000040eb00bb
:1091d000604798000040eb00504798000040eb00cb
:1091e000404798000040eb00304798000040eb00fb
:1091f000204798000000eb00000f78000040eb00d3
:1092000040479800100037004e4090000080fb005f
:109210007400b900ea004000a08f200000804000e8
:10922000904078000e50900080cf500003003a002c
:1092300010002000300f9800820137004e4090004f
:109240000040e800404798004e4090000004e000d5
:10925000edff32000040eb0040479800030037006c
:109260004e4090000040e800404798004e4090007b
:109270000004e00009003a004e4090000080fb002e
:109280007400b900ea004000a08f20000080400078
:10929000104078000004e000f1ff3a004e409000da
:1092a000e14f500003003a008000eb00310f9800be
:1092b0006401370080488000700798000000eb00d0
:1092c000400798004e4090008081fb00ce00900047
:1092d0007e00900000804000640040001041780053
:1092e0007418b90080007800809020000080400051
:1092f000024878002c013700ce0090007e009000dc
:10930000008040000000e80010407800e44f50006a
:109310001d013a00ce0090007e00900000804000c9
:109320006500400010407800e34f500046003200d6
:10933000ce0090007e00900000804000650040005c
:10934000104078000004e0000f013a003e003700b2
:109350002e4090000080fb004300dd00e60040004e
:10936000a08e200000804000100078000000d10096
:10937000614060000004e000300032002e409000a8
:109380000080fb00c300dd00a08e200000804000b4
:1093900010417800ce0090007e00900000804000d8
:1093a0006500400010407800804f510023003a00d3
:1093b0002e4090000080fb00c300dd00a08e200046
:1093c0000080400010419000ce0090007e00900090
:1093d000008040006600400010407800804f51003f
:1093e00016003a002e4090000080fb004300dd0094
:1093f0008080e800a08e20000080400010417800ae
:10940000ce0090007e009000008040006700400089
:1094100010407800804f510008003a004e40900004
:109420000080fb007400b9008000780020902000cc
:109430008080400010c0b300904098002e40900003
:109440000040e800204798002e409000e14f500077
:10945000bfff36000040eb00204798004e409000d0
:109460000080fb007400b900e8004000a08f2000dd
:1094700000804000104090000004e000c200320074
:10948000a00020002de50700000f78001e00e0007e
:1094900003003a008000eb00310f9800e90037002c
:1094a0003e4090000040e80030479800204980008e
:1094b0000000e00005003a001e0078002049880006
:1094c0009e0078003149880007003700304980004d
:1094d0001e0878001e00780030498800314980005d
:1094e0000000eb008008780032498000ce00900038
:1094f0007e009000008040000080e800104078006e
:1095000000499800ce0090007e009000008040004e
:10951000104078008080fb004e0090000100400069
:1095200040079800ce0090007e0090000080400030
:109530000000e8009040780010c2b30080cf5000d7
:1095400091003a00ce0090007e0090000080400024
:1095500065004000104078000004e00011003a006f
:109560000000eb00500798004e0090007400b90016
:1095700080007800409020008080400050c5b300fb
:10958000904098004e0090007400b9008000780070
:10959000609020008080400000c6b30080487800c2
:1095a00079003700100020005007980033498000f0
:1095b000ce0090007e0090000080400067004000d8
:1095c000104078000081fb00ce0090007e009000eb
:1095d0000080400068004000104078000080fb00e0
:1095e0004800dd0000007100900198000040eb0091
:1095f000604798000040eb0050479800ce00900074
:109600007e00900000804000104078008080fb00c9
:109610004e0090000100400040079800ce009000ee
:109620007e009000008040000000e80010407800bc
:10963000e54f500027003a00ce0090007e009000d9
:10964000008040006300400010407800e34f50006d
:1096500020003a00ce0090007e0090000080400084
:109660000080e800104078000004e00009003d00a0
:109670006e4090000004e00006003a00ce0090002a
:109680007e009000008040000080e800904078005c
:1096900061479800ce0090007e009000008040005e
:1096a0000080e800104078000004e0000900350068
:1096b0005e4090000004e00006003a00ce009000fa
:1096c0007e009000008040000080e800904078001c
:1096d000514798006e4090000004e00003003a00fb
:1096e0005e4090000004e000270032004e409000f1
:1096f0000080fb007400b9008000780040902000da
:10970000008040008e509000014878003049800071
:10971000ee4090006140980030498000de409000ab
:109720007140980033498000ce0090007e00900088
:109730000080400064004000104078000081fb0081
:10974000ce0090007e009000008040006500400048
:10975000104078000080fb004800dd000000710030
:10976000a001980032498000ce0090007e00900059
:1097700000804000660040001040780010499800ca
:109780001000200060079800ce0090007e0090003e
:1097900000804000104078008080fb004e00900068
:1097a0000100400040079800fe009000214090001a
:1097b0000081fb00314090000080fb004800dd008c
:1097c00002007000800078004e009000808f5000f2
:1097d000c9fe3e004e4090000080fb007400b900be
:1097e000ee004000a08f20000080400090407800f4
:1097f0003e40900080cf5000020032000000eb009d
:10980000600798006e0090000000e0000b0032003e
:109810004e4090000080fb007400b900800078008a
:10982000609020008080400000c1b3008048780034
:1098300010002000300f9800020037008000eb007d
:10984000310f98003e0890000080fa0000000600ea
:109850000600fa00404798000040eb00004f7800f7
:10986000010037001e4fe8001e04e00009003a0026
:109870001e80fb007400b900ea004000a08f2000a9
:1098800000804000904078004e40900080cf500013
:10989000f4ff3a001e04e00025003a004044800036
:1098a00078e407000000eb00404488001e80fb00c5
:1098b0007400b900e4004000a08f20000080400048
:1098c000100078006fe407001e80fb007400b900f0
:1098d00080007800e08f2000808040000000eb00d6
:1098e000800878000f003700204980009000780041
:1098f000110798002049800062e407000000eb0097
:1099000020498800304980005ee407000000eb0039
:10991000304988001e0090002049880020498000be
:1099200030498800204980000000e000eeff3a0046
:109930000080fa00000006000200fa00004f7800e4
:109940001e80fb007400b900e8004000a08f2000da
:1099500000804000100078000000d10061406000ed
:109960000004e000080032001e80fb007400b90013
:1099700080007800609020008080400000c4b30028
:109980008048780018003700208d2000900190005a
:109990001e80fb007400b900ea004000a08f200088
:1099a00000804000104078006022b8000001eb0009
:1099b00021132000030001009e81fb001e80fb009c
:1099c0007400b900ec004000a08f2000008040002f
:1099d000104190007418b900800078006090200059
:1099e00000804000024878000080fa000000060075
:1099f0003e00fa00881f7800101798002117980081
:109a000032179800036f98000000eb00500f980089
:109a10000000eb00400f98000000eb00300f9800b2
:109a20000000eb00200f98000000eb00100f9800e2
:109a30000000eb00000f98000000eb00700798009a
:109a40000040eb00404f98000000eb0050079800ea
:109a50000000eb00400798000000eb003007980082
:109a60000000eb00200798000040eb002047980022
:109a70000040eb00104798000040eb00004f7800da
:109a80001e1090000000e000030032002e10900035
:109a90000000e00003003a0020002000401f980072
:109aa000ec043700ef0407000e68900057e8b70099
:109ab000ae109000410f98004e09900012418800ae
:109ac0009e119000330f9800bc0037003e089000b4
:109ad000904078007c004700014878007c004700f7
:109ae0001000780063406000004f78007c00470061
:109af0001000780063006000e30f500002003a009d
:109b000040c0b300004f78001e80fb00800078004a
:109b10003e089000008040000000e800300f9800f0
:109b20009e80fb004e089000010050000000e900fc
:109b3000400f98007c004700100078004200de00d3
:109b4000634060000080fb00301f98003e1b9000c7
:109b5000e10f530038003200be1b9000e28f53002b
:109b60005f0032003e1c90000800e000010032005f
:109b7000920037007c004700100078004400de00af
:109b80006f4060000080fb00201f98002e1890009e
:109b9000e80f500089003500ae189000e98f5000a2
:109ba000210034002e199000ea0f51000700320006
:109bb000ae199000eb8f51001b0032002e1b90005d
:109bc000ec0f53000f0032007c00370047c8bf0085
:109bd0000040e80047e8b70046c8bf000040e80082
:109be00046e8b70061842000914078004dc8bf006e
:109bf00080cf50007100360046c8bf004de8b70066
:109c00006e00370046c8bf000040e90046e8b700d4
:109c100046c8bf00e14f400068003a003000200015
:109c2000200798006500370050c8bf000040e800da
:109c300050e8b700610037007c0047001000780052
:109c40004400de006f4060000080fb00101f9800a1
:109c50009e1b9000ea8f53000b0032001e1c9000e8
:109c6000eb0f5400130032001e189000e80f500054
:109c7000010032005100370051c8bf000040e80029
:109c800051e8b7004d0037004cc8bf000040e80065
:109c90004ce8b700c1842000914078004ec8bf0056
:109ca00080cf5000450036004cc8bf004ee8b700da
:109cb000420037004cc8bf000040e9004ce8b70044
:109cc000c1842000914078004ec8bf0080cf500072
:109cd0003a00360040002000200798003700370087
:109ce0007c004700100078004400de006f406000f8
:109cf0000080fb00001f98008e189000e58f500038
:109d00000d003c000e199000e40f510028003d00aa
:109d10008e199000e28f510021003c000e1b900034
:109d2000e10f530012003d008e1b90000700e00081
:109d30000b003200210037000e1c9000e70f54008a
:109d40000f0032000e189000e70f50001b00350086
:109d50008e189000e98f500018003c000c0037006e
:109d600056c8bf000040e80056e8b70013003700af
:109d7000204280000000e800204288000f003700e9
:109d800054c8bf000040e80054e8b7000b0037009b
:109d9000f04180000000e800f04188000700370033
:109da000b04180000000e800b041880003003700a7
:109db000a04180000000e800a04188004e0890000b
:109dc0000000e00041ff3a002e0090000000e0009b
:109dd000030032002e019000421f98001d0437003e
:109de00046c8bf000004e00003003200530020001a
:109df000431f98001704370047c8bf00e14f5000c9
:109e000003003a0066002000461f98001104370046
:109e100050c8bf000004e00003003a0077002000b3
:109e2000471f98000b04370020428000610060004b
:109e30000004e0000300320088002000481f980062
:109e400004043700f0418000610060000004e0007d
:109e50000300320090002000401f9800fd033700ef
:109e6000a0418000610060000004e00003003200b7
:109e7000a1002000411f9800f603370061852000f3
:109e800091407800204280000000d10000c04000d6
:109e900056e8b7004185200091407800f0418000ed
:109ea0000000d10000c0400054e8b700b14180007c
:109eb000a04180000000d10000804000b041880037
:109ec00047c8bf000080fb006e00b90000017800a9
:109ed00050c8bf008080fb00e00220000088b9006d
:109ee0000001410056c8bf000080fb006a00b900b5
:109ef0008000780051c8bf000080fb004300dd00f7
:109f000000804000800141004ec8bf000080fb007f
:109f10004201dd00b141800054c8bf000080fb0059
:109f20000080400000004100c200dd004dc8bf00bd
:109f30000080fb00008040000000400000804100e5
:109f4000500f9800404480000000e0000400320000
:109f500040448000cbe207000000eb004044880052
:109f60005e08900075e2070040448800404480008d
:109f70000000e00003003a0012002000421f980099
:109f8000b403370043448000230f98002e0890004c
:109f9000c043880047c8bf000080fb006e00b900c6
:109fa000800078002e08900001004000200f9800eb
:109fb0002e089000f043880050c8bf008080fb004e
:109fc000e00220000088b900800078002e08900090
:109fd00001004000200f98002e08900000448800e7
:109fe00051c8bf000080fb004300dd008000780006
:109ff0002e08900001004000200f98002e089000cd
:10a000002044880056c8bf000080fb006a00b900e9
:10a01000800078002e08900001004000200f98007a
:10a020002e0890001044880054c8bf000080fb0038
:10a030004300dd00800078002e0890000100400001
:10a04000200f98002e089000d0438800b041800077
:10a050004300dd00800078002e08900001004000e1
:10a06000200f98002e0b9000364488004dc8bf008a
:10a070000080fb0000004000800078002e08900067
:10a0800001004000200f98002e089000e043880057
:10a0900074030700c7438000170f98001e09900043
:10a0a0006000b8000089be009e0890000040eb00f0
:10a0b000b04898009e0890000040eb00804898004f
:10a0c0009e0890000040eb00e04098009e08900041
:10a0d0000040eb00c04898009e0890000040eb0054
:10a0e000a04898009e0890000040eb00904898001f
:10a0f0009e0890000040eb00f04098009e08900001
:10a100000000eb00a000980008448000080f9800b1
:10a110008e0890000000eb00b00098008e089000c0
:10a120000000eb00900098008e0890000000eb000b
:10a13000a00098008e0890000000eb0080087800d6
:10a140002e109000400f98009e109000310f980044
:10a15000030337003e089000904078007c004700e1
:10a16000014878007c0147006000b80010019800a9
:10a17000210198007c0047001000780063406000d7
:10a18000004f78007c0047001000780063006000fa
:10a19000e30f500002003a0040c0b300004f7800c7
:10a1a0003e0890000000e800300f98000040eb00ef
:10a1b000204798001f0037003e08900010417800ab
:10a1c000124798003e0890000000e800300f980009
:10a1d0007c00470010029000a00290001e409000fa
:10a1e0000081fb00030020002e4090000080fb0057
:10a1f0004300dd000203be00000478000804e9000b
:10a20000030033000603430087834b00fbff370046
:10a210000600be0000007200818072007c014700d1
:10a2200010019800210198002e4090000040e800a5
:10a23000204798002e4090009e4f5000deff3900ce
:10a240009e80fb004e089000010050000000e900d5
:10a25000400f98007c004700100078004200de00ac
:10a26000634060000080fb00701798007e10900033
:10a27000e10f500027003200fe109000e28f5000e6
:10a28000e50032007e1190000200e0000100320083
:10a29000ad0237007c004700100078004400de006b
:10a2a0006f4060000080fb0060179800ee11900086
:10a2b000e88f5100a40235006e139000e90f53009f
:10a2c0000a003400ee139000ea8f53000b003200b6
:10a2d0006e149000eb0f5400040032006e109000da
:10a2e000ec0f500008003200970237007c00470056
:10a2f0008603070020079800930237007c00470080
:10a300001f030700900237007c004700620307002c
:10a310008d0237007c004700100078004400de000a
:10a320006f4060000080fb006101b900521f98007f
:10a33000631f9800b0002000010020005e1b900009
:10a34000ee1b9000800f5300818f5b007e023e0069
:10a350005e189000ee189000006001000b003700be
:10a360000f003700160037001d00370024003700ab
:10a370002b003700740237002f00370038003700f9
:10a380007d0037008a003700960037007c004700c8
:10a39000a000900010009000c04288006a023700c0
:10a3a0007c0047003e0407007c004700a0009000ae
:10a3b00010009000d0428800e1428800620237001d
:10a3c0007c004700360407007c004700a000900096
:10a3d00010009000f0428800014388005a023700c4
:10a3e0007c0047002e0407007c004700a00090007e
:10a3f000100090001043880021438800520237006b
:10a400007c004700260407007c004700a000900065
:10a410001000900030438800414388004a02370012
:10a420007c004700a000900010009000504388007e
:10a4300061438800440237007c004700a000900080
:10a440001000900075e8b70075c8bf000004e00078
:10a450003d023a00f0002000200798003a02370041
:10a460007c004700a000900010009000e00f50001a
:10a47000e08f58003d0032000040eb00404f980054
:10a48000030037004e4890000040e800404f98001d
:10a4900011852000914078004e48900080cf5000f8
:10a4a0000d003600014480004e4890000080fb0003
:10a4b0004300dd0000804000100078006101b8001a
:10a4c0007c004700a000900010009000800f510019
:10a4d000818f5900ebff3a001185200091407800f0
:10a4e0004e48900080cf500018003a000144800090
:10a4f00012852000124178000280fb004300dd003d
:10a5000000804000700798000240e80051e8b70062
:10a510007c004700a00090001000900080007800b0
:10a520007e00900001087800fe009000800020006e
:10a5300090009800fe00900080002000a00098008d
:10a54000fe00900080002000b00098007c004700d2
:10a55000a00090001000900074e8b7004e489000f2
:10a560000080fb0090438800f701370000012000c5
:10a5700020079800f40137007c004700a0009000fd
:10a5800010009000e00f5000e08f580005003200ee
:10a590007c004700a00090001000900076e8b70013
:10a5a000e90137001001200020079800e60137007c
:10a5b000e1438000c2842000124178000280fb0049
:10a5c0004500dd0000804000818520000f0009006b
:10a5d000311878000002b1000240e8004ce8b700f2
:10a5e000d9013700e14380004cc8bf000040e900ba
:10a5f0004ce8b7004cc8bf000080fb004500dd0000
:10a6000000804000828520000f000900301978008a
:10a610000002b100cc0137007c0047001000780038
:10a620004400de006f4060000080fb00501798007f
:10a63000de119000e48f5100210132005e13900082
:10a64000e40f530011003c00de139000e18f530033
:10a650004b0032005e149000e10f540004003c00f7
:10a660005e1090000000e00019003200b6013700d3
:10a67000de109000e28f50009d0032005e119000cd
:10a68000e30f5100fb003200af013700de119000f4
:10a69000e78f5100520132005e139000e70f530024
:10a6a00004003c00de139000e58f530028013200c7
:10a6b000a50137005e149000e80f54005b013200e2
:10a6c0005e109000e90f50007c0132009e013700bf
:10a6d0002344800052852000124178000280fb0054
:10a6e0006a00b90000804100300798000240e8008d
:10a6f00055e8b700be0090000000eb00800878002d
:10a700007c0047001000780063006000e30f5000f9
:10a7100011003a007c004700a0009000100090005b
:10a720004008de0001002000800078003e0090001c
:10a73000110098007c004700a000900010009000dd
:10a7400080007800f00f2000808060003e009000c4
:10a75000210098007c013700c14280003e0090003b
:10a76000110098007c004700a000900010009000ad
:10a77000800078003e0090002100980072013700b0
:10a78000604180000000e0003d0032002344800072
:10a7900052852000124178000280fb006a00b90057
:10a7a00000804100300798000240e80055e8b700fb
:10a7b000be00900010002000800878007c00470058
:10a7c0001000780063006000e30f500011003a00b1
:10a7d0007c004700a0009000100090004008de00c0
:10a7e00001002000800078003e00900011009800d9
:10a7f0007c004700a00090001000900080007800ce
:10a80000f00f2000808060003e0090003100980032
:10a8100009003700c14280003e00900011009800fe
:10a820007c004700a000900010009000800078009d
:10a830003e00900031009800200120002007980081
:10a84000014280003e009000410098003e009000d0
:10a85000c00090003e00900030009000808f5000bb
:10a860000200310030012000200798000000eb00ba
:10a87000604188000000eb00704188003201370021
:10a880007c0047001000780063006000e30f500078
:10a890000e003a007c004700a000900010009000dd
:10a8a0004008de0001002000c04188007c00470015
:10a8b000a00090001000900080007800f00f2000b1
:10a8c000008060001042880006003700c04280000f
:10a8d000c04188007c004700a0009000100090005c
:10a8e00010428800100020007041880016013700d7
:10a8f000704180000000e0004200320023448000ec
:10a9000052852000124178000280fb006a00b900e5
:10a9100000804100300798000240e80055e8b70089
:10a92000be00900010002000800878007c004700e6
:10a930001000780063006000e30f500011003a003f
:10a940007c004700a0009000100090004008de004e
:10a9500001002000800078003e0090001100980067
:10a960007c004700a000900010009000800078005c
:10a97000f00f2000808060003e00900041009800b1
:10a9800009003700c14280003e009000110098008d
:10a990007c004700a000900010009000800078002c
:10a9a0003e009000410098003e0090009000900012
:10a9b000c0418000808f5000020032002001200042
:10a9c00020079800114280003e009000310098005e
:10a9d0003e009000c00090003e00900030009000cb
:10a9e000808f5000020031003001200020079800c5
:10a9f0000000eb00604188000000eb00704188001f
:10aa0000d10037007c004700100078006300600030
:10aa1000e30f50000e003a007c004700a0009000b9
:10aa2000100090004008de0001002000c0418800b6
:10aa30007c004700a000900010009000800078008b
:10aa4000f00f200000806000004288000600370000
:10aa5000c0428000c04188007c004700a0009000f8
:10aa60001000900000428800100020006041880023
:10aa7000b5003700d1438000828420001241780065
:10aa80000280fb004300dd0000804000500798007a
:10aa90000240e80048e8b700de0090000000eb004c
:10aaa000800878007c004700a00090001000900013
:10aab000800078005e00900011009800a20037002e
:10aac000204180000000e0001a003200d1438000e5
:10aad00082842000124178000280fb004300dd00e8
:10aae00000804000500798000240e80048e8b700a6
:10aaf000de00900010002000800878007c004700f5
:10ab0000a000900010009000800078005e0090008f
:10ab100021009800814180005e0090003100980083
:10ab20000000eb00304188000000eb00204188006d
:10ab3000850037007c004700a000900010009000c6
:10ab40009041880010002000304188007e003700ce
:10ab5000304180000000e0001a003200d143800044
:10ab600082842000124178000280fb004300dd0057
:10ab700000804000500798000240e80048e8b70015
:10ab8000de00900010002000800878007c00470064
:10ab9000a000900010009000800078005e009000ff
:10aba00031009800914180005e00900021009800e3
:10abb0000000eb00304188000000eb0020418800dd
:10abc000610037007c004700a0009000100090005a
:10abd0008041880010002000204188005a00370082
:10abe0001144800032852000124178000280fb0071
:10abf0004300dd0000804000400798000240e8006c
:10ac000053e8b700ce0090000000eb008008780009
:10ac10007c004700a00090001000900080007800a9
:10ac20004e0090001100980047003700404180001e
:10ac30000000e0001a00320011448000328520003c
:10ac4000124178000280fb004300dd0000804000dc
:10ac5000400798000240e80053e8b700ce0090009b
:10ac600010002000800878007c004700a0009000c1
:10ac700010009000800078004e00900021009800a5
:10ac8000d14180004e009000310098000000eb00a0
:10ac9000504188000000eb00404188002a00370046
:10aca0007c004700a000900010009000e041880068
:10acb00010002000504188002300370050418000e0
:10acc0000000e0001a0032001144800032852000ac
:10acd000124178000280fb004300dd00008040004c
:10ace000400798000240e80053e8b700ce0090000b
:10acf00010002000800878007c004700a000900031
:10ad000010009000800078004e0090003100980004
:10ad1000e14180004e009000210098000000eb000f
:10ad2000504188000000eb004041880006003700d9
:10ad30007c004700a000900010009000d0418800e7
:10ad400010002000404188002e0090000000e0002c
:10ad500003003200ae009000411f98003d00370014
:10ad60004e0890000000e000fafc3a0010c0b3006a
:10ad70002047980030003700014480002e409000aa
:10ad80000080fb004300dd000080400010009000c8
:10ad9000e80f500007003a00014480002e40900068
:10ada0000080fb004300dd00808040000000eb00dd
:10adb00090009800014480002e4090000080fb002d
:10adc0004300dd000080400020009000e80f5000ac
:10add00007003a00014480002e4090000080fb00f4
:10ade0004300dd00808040000000eb00a0009800e0
:10adf000014480002e4090000080fb004300dd00f5
:10ae00000080400030009000e80f500007003a003a
:10ae1000014480002e4090000080fb004300dd00d4
:10ae2000808040000000eb00b00098002e409000b1
:10ae30000040e800204798001185200091407800ec
:10ae40002e40900080cf5000cbff3e002e0190009e
:10ae5000421f98004e1890004f0478000080fa00be
:10ae6000000006000000fa000040eb0046e8b700d2
:10ae700010c0b30047e8b7000000eb00a041880015
:10ae80000000eb00b04188000040eb004ce8b70048
:10ae90000040eb004de8b7000040eb004ee8b70083
:10aea0000040eb0050e8b70010c0b30051e8b70015
:10aeb0000000eb00f04188000040eb0054e8b700d0
:10aec0000040eb0056e8b7000000eb00204288008d
:10aed0000040eb0055e8b7000000eb00204188007f
:10aee0000000eb00304188000000eb00404188008a
:10aef0000000eb00504188000000eb00604188003a
:10af00000000eb00704188006000b800f04288004b
:10af1000014388006000b800d0428800e142880008
:10af20006000b80030438800414388006000b800ea
:10af300010438800214388000040eb0076e8b7000a
:10af40000040eb0074e8b7000000eb00904388007d
:10af50000040eb0075e8b7006000b800704388005f
:10af6000814388006000b800504388006143880036
:10af70000000eb00c04288000080fa0000000600dc
:10af80000600fa00200798007184200091407800a4
:10af90000180fb00000f78000140e80047e8b7009f
:10afa000c24380001e0078006e00b900000041001e
:10afb000100798002e009000a00090001000900054
:10afc0001e0190000089be0091842000914078000d
:10afd0001e0090006140980051852000914078004b
:10afe00049c8bf0080c050001e009000714098000a
:10aff00055c8bf0049e8b70021852000914078007e
:10b000001e009000414898000040eb0052e8b70055
:10b010009e0090000040eb00b0489800c1428000c4
:10b020001e009000210098000185200091407800ca
:10b030001e00900001489800f184200091407800a3
:10b040001e00900021489800c24380004fc8bf00f6
:10b050000080fb006e00b900800041001e007800f7
:10b06000b04898003144800062842000124178008a
:10b070000280fb00808040004fc8bf0080487800fd
:10b080000240e80046e8b7001e0078004fe8b7002d
:10b090000080fa00000006000600fa002007980071
:10b0a000c24380004fc8bf000080fb006e00b900a3
:10b0b00000004100100798000185200091407800b1
:10b0c0001e0090000048900080c050001e009000bc
:10b0d000114898003144800046c8bf000040e90094
:10b0e00046e8b70046c8bf000080fb000080400073
:10b0f000104f78004fc8bf0052e8b7001e407800dc
:10b100004fe8b7000080fa00000006000c00fa00cb
:10b11000300798000000eb00200798000000eb00cb
:10b12000100798000000eb00000f78003e00900030
:10b130000000e00003003a002000200050079800c3
:10b14000d4003700d4428000e542800075c8bf00bb
:10b150000081fb0010002000010020008201780027
:10b160008301e900030033000000400081804800b3
:10b17000fbff3700800f5200818f5a00030035001b
:10b18000c000200050079800c2003700f442800041
:10b190000543800075c8bf000081fb00100020003f
:10b1a00001002000820178008301e90003003300e0
:10b1b0000000400081804800fbff3700800f5200f4
:10b1c000818f5a0003003500d000200050079800fe
:10b1d000b0003700d2428000e3428000f04280009d
:10b1e00001438000800f5100818f5900030034001b
:10b1f000e100200051079800a60037007041800050
:10b200000000e00003003a00604180000000e00020
:10b210000300320083002000530798009d00370090
:10b22000504180000000e00003003a0040418000ef
:10b230000000e0000300320090002000500798005a
:10b2400094003700304180000000e00003003a0025
:10b25000204180000000e00003003200a100200037
:10b26000510798008b003700f243800003852000cf
:10b27000934178008380fb00e00220000088b90041
:10b2800000004100200798000340e80050e8b700a4
:10b290003e009000a0009000100090002e01900051
:10b2a00020119800311198002e0090000080e800d5
:10b2b000838520000f000900331878000002b100d8
:10b2c000f1842000914078002e00900031609800b9
:10b2d00091842000914078002e0090000168980031
:10b2e00055c8bf0049e8b70051852000914078005b
:10b2f0002e0090000068900080c050002e0090004a
:10b3000011689800b1842000914078002e009000d0
:10b310002168980053c8bf004be8b7003185200072
:10b32000914078002e0090002068900080c050006e
:10b330002e00900031689800a18420009140780090
:10b340002e0090004168980048c8bf004ae8b70046
:10b3500081842000914078002e0090004068900089
:10b3600080c050002e009000516898000144800079
:10b37000904380004300dd000080400010079800eb
:10b3800075c8bf008080fb0076c8bf000080fb004e
:10b390000088b900000f78003e009000100078008f
:10b3a0004400de006f4060000080fb004007980012
:10b3b0004e009000e90f500015003200ce009000c2
:10b3c000eb8f500004003200ce019000e88f510056
:10b3d0001d0032002a003700ae009000200020003f
:10b3e000800878001e0090003000900080407800b7
:10b3f0002e009000216098001e0090003000900008
:10b400009e0040001e009000310098001f00370091
:10b41000ae00900010002000800878001e00900010
:10b4200020009000804078002e009000216098005d
:10b430001e009000200090009e0040001e00900022
:10b440002100980011003700ae0090000000eb00d2
:10b45000800878001e009000100090008040780066
:10b460002e009000216098001e00900010009000b7
:10b470009e0040001e00900011009800030037005d
:10b48000ae00900030002000800878000000eb0043
:10b49000500798005e0090000080fa00000006004f
:10b4a0000400fa00100798000040eb0010479800d5
:10b4b0001e0090001000780063406000004f78008c
:10b4c0001e04e000230032001e00900010007800ef
:10b4d00063006000e30f500002003a0040c0b30078
:10b4e000004f78001e80fb000000e9009e009000e5
:10b4f0000080e8000100400090407800114798006b
:10b500001e4090000004e00012003d000e003700d5
:10b510001e00900010019000a00190001e80fb0012
:10b52000c300dd00f00f20000100dd00cf80de0051
:10b5300000007100818071001e01900010019800d0
:10b54000210198001e4fe80030c0b3009e4f10004c
:10b55000efff36000080fa00000006001c00fa0031
:10b560006007980071079800020f9800130f980069
:10b57000240f98000040eb00305f98006e009000b0
:10b580000000e00002003a0011c0b300315f9800f3
:10b590000041eb00225f98001e0890000000e000d0
:10b5a00002003a0010c0b300205f9800be5890001f
:10b5b0002e59900002c070000004e0000300320029
:10b5c0000000eb00400f9800a50037006e009000cf
:10b5d00080689000214798000000eb004007980029
:10b5e0000040eb00004f78009700370022448000b5
:10b5f0002e4090000080fb006a00b900000041006e
:10b60000500798002e4090000040e8002047980026
:10b610007e0090000000e000050032005e00900017
:10b62000900090007e009000808f500003003a0050
:10b6300012002000320f9800020037000000eb00db
:10b64000300f9800be089000210798005e0090001f
:10b65000100078000000e000490032005e00900019
:10b66000b00090000e089000808f500038003e001f
:10b670005e009000c00090000e089000808f500087
:10b68000330039001e0890000000e000080032007e
:10b690005e009000b00090000e0890008100500005
:10b6a0004e009000808040001e0890000108780045
:10b6b0002e0890000000e0001f0032001e80fb00fa
:10b6c0008000e8006e009000106890000080fb0091
:10b6d000808f500015003a005e009000c00090007e
:10b6e0000e089000808f500010003a006e0090000d
:10b6f000806090004e00900000c0500010479800fd
:10b700001e409000e14f5000040036002e089000cb
:10b710001e4190000248780007003700ae089000f4
:10b7200010c0b3008048780003003700ae089000d6
:10b7300010c0b300804878002e0090000000e000a8
:10b740000300320010002000400f98004400370032
:10b750005e009000c00090005e00900030009000fd
:10b76000008050000000e80030079800ce009000f4
:10b770003e009000008040004007980031003700f4
:10b780005e009000a00090000e089000808f500096
:10b7900029003a001e0890000000e000030032007b
:10b7a0001e089000ce009000010878002e0890003e
:10b7b0000000e0001a0032001e80fb008000e8005c
:10b7c0006e009000106890000080fb00808f500099
:10b7d00010003a006e009000806090004e009000d3
:10b7e00000c05000104798001e409000e14f5000ec
:10b7f000040036002e0890001e4190000248780098
:10b8000007003700ae08900010c0b30080487800f1
:10b8100003003700ae08900010c0b30080487800e5
:10b820002e0090000000e000030032001000200015
:10b83000400f98000a0037004e0090000000e8001a
:10b84000400798001e4fe8006e00900010689000be
:10b850009e4f500065ff3e008000eb00410f9800b6
:10b860004e0890000080fa00000006000e00fa006a
:10b87000004f7800110798002207980034079800bd
:10b88000450798001e009000600798006e00900029
:10b89000f00f50002c0032006e009000f00f5000ae
:10b8a0000a003e006e009000ed0f500014003200c0
:10b8b0006e009000ee0f50001b0032006e009000f2
:10b8c000e80f50001b003200380037006e00900077
:10b8d000f20f5000260032006e009000f20f500070
:10b8e0001e0039006e009000f30f5000250032005a
:10b8f0006e009000f40f5000270032002b0037003c
:10b900002e00900010409000e64f400003003e00e3
:10b910001000200050079800260037002060290002
:10b92000d7080700210037001000200050079800ba
:10b9300020003700f0632900d10807001000200024
:10b94000500798001b00370020672900cc0807002b
:10b95000100020005007980016003700606a290088
:10b96000c70807001000200050079800110037009a
:10b97000a06d2900c20807001000200050079800a1
:10b980000c00370090712900bd080700100020004e
:10b99000500798000700370080742900b808070096
:10b9a0001000200050079800020037000000eb0054
:10b9b000500798005e0090000080fa00000006002a
:10b9c0000400fa00616a20009140780000ccb300c6
:10b9d00000c06000a040b300a6e6b700116d2000d3
:10b9e0009140780000ccb30000c060005040b3002c
:10b9f000d1e6b70020302300103a88000000eb00a9
:10ba0000203a8800000c2000c01688008208070039
:10ba1000f03f2000103088003038280000308800c7
:10ba200010002000603088009007070000003700f9
:10ba30000ddf0700e1ef07007d010700d04880001f
:10ba4000100798001e009000e30f500041003200e4
:10ba50001e009000e30f500007003e001e00900003
:10ba6000e10f5000220032001e009000e10f500054
:10ba700032003e000a0037001e009000e50f500023
:10ba80007f0032001e009000e50f50004200390098
:10ba90001e009000e60f500089003200e4ff3700de
:10baa000f1de0700c5ef0700004980000000e0005c
:10bab00007003a00d4070700b30707000077290002
:10bac00011c0b30081030700100020000049880066
:10bad000330507000000e000d5ff32001000200011
:10bae000d04888000000eb00f0488800d0ff370005
:10baf00020002000d0488800f04880000000e000ce
:10bb00000c003a00c00707009f07070010782900c3
:10bb100011c0b3006d0307002079290021c0b300d4
:10bb20006a03070010002000f04888000000eb00c6
:10bb30000049880090040700bdff37001805070082
:10bb40000000e000baff3a000000eb00d048880097
:10bb5000b7ff3700208c2000a0019000208c20002f
:10bb60001000900000417800c189200091407800c9
:10bb7000208c2000100078001d0507000004e00064
:10bb800002003a0040002000d0488800b6de0700de
:10bb90008aef0700a6ff3700d18c2000b08c200070
:10bba000390507000000e000a1ff3200cbc8bf004c
:10bbb0000004e00006003a00cdc8bf008080fb0012
:10bbc000208c200010009000808f50000c0032006c
:10bbd000ccc8bf000040e800cce8b700cbc8bf002d
:10bbe000e94f50000300360070002000d048880064
:10bbf0008fff370020002000d04888008cff3700de
:10bc00000040eb00cce8b700100020007046880030
:10bc100020002000d0488800f0488000e10f50004c
:10bc200014003a000040eb00004f78000c00370091
:10bc3000208c2000a00090001e80fb0000804000af
:10bc4000104078000004e000040032006e07070096
:10bc50004d0707000000eb00f04888001e4fe80089
:10bc60001e80fb00218c200091009000810f50006d
:10bc7000efff390037000700270007006cff37008f
:10bc8000a18c2000504480000041780092c8bf0081
:10bc900064448000810178008040780004007800ce
:10bca000e60407000004e00002003a006000200003
:10bcb000d04888006cde070040ef07005cff3700cb
:10bcc000d18c2000b08c2000ef0407000000e000c1
:10bcd00057ff3200cbc8bf000004e000090032006b
:10bce000ccc8bf000040e800cce8b700cbc8bf001c
:10bcf000e94f50004eff360070002000d048880009
:10bd00004bff37000040eb00cce8b70020002000dc
:10bd1000d048880046ff37000000fa0070468000d7
:10bd2000e10f500009003a000000eb007046880067
:10bd3000e04880000000e0000400320050002000d5
:10bd4000d04888000000eb00e04888000080fa003e
:10bd5000000006000400fa00208c200090009000f3
:10bd6000208c20002000900043892000828a20003f
:10bd700002060700208c200090009000208c2000fc
:10bd800020009000e3892000028b2000fb050700c3
:10bd90000040eb00104798005b0037001e40900009
:10bda0008080fb00008b2000008040001040780065
:10bdb0000004e000510032001e4090008080fb0033
:10bdc000008b2000008040009040780090c3b300ba
:10bdd00080cf500016003a0022c9bf008040eb001f
:10bde000314798000004e00002003a0010c0b300a0
:10bdf000304798003e40900022e9b7001000200034
:10be0000e048880022c9bf006140600061406000d6
:10be100000414000a18c200091407800d0cfb300b9
:10be200000c0600002407000cae8b700330037006d
:10be30001e4090008080fb00008b200000804000ae
:10be40009040780030c5b30080cf500015003a0014
:10be500023c9bf008040eb00214798000004e000a8
:10be600002003a0010c0b300204798002e40900016
:10be700023e9b70010002000e048880023c9bf0074
:10be80006140600061416000a18c20009140780019
:10be9000e0cfb30000c0600002407000cae8b70005
:10bea000160037001e4090008080fb00008b2000b1
:10beb0000080400010407800340007000000e000df
:10bec0000e003a001e4090008080fb00008b200096
:10bed00000804000104078007b000700004f780091
:10bee0001e4090008080fb00008b200000804000fe
:10bef000904078001e407800960107001e40900098
:10bf00000040e800104798001e409000e54f5000a8
:10bf1000a2ff3600030007004d0007000080fa0072
:10bf2000000006000200fa000040eb00004f78001d
:10bf3000110037001e81fb009e80fb00608b2000fb
:10bf40000080400090407800c08b2000000041003d
:10bf5000014878001e81fb009e80fb00008b2000c2
:10bf60000080400090407800608b2000000041007d
:10bf7000014878001e4fe80050c0b3009e4f1000eb
:10bf8000ecff36000080fa00000006000600fa0010
:10bf9000204798000040eb00004f78001c0037005d
:10bfa0009e80fb00608b2000008040009040780065
:10bfb0002e40900080cf500014003a000040eb006b
:10bfc000004f78000b0037009e80fb00c08b2000e4
:10bfd00000804000904078002e40900080cf5000bc
:10bfe00003003a000000eb00200798000d00370026
:10bff0001e4fe80050c0b3009e4f1000f2ff360005
:10c000001000200020079800060037001e4fe800af
:10c0100050c0b3009e4f1000e1ff36000000eb005f
:10c02000200798002e0090000080fa000000060013
:10c030000000fa00da0307000000e00002003a0006
:10c040000000eb00d04888000080fa0000000600e5
:10c050000200fa000040eb00004f780006003700b5
:10c060009e80fb00008b2000808040000040eb00a1
:10c07000804878001e4fe80050c0b3009e4f10006b
:10c08000f7ff36000040eb00004f78000700370054
:10c09000208c2000a00090001e80fb0080804000cb
:10c0a0000040eb00804878001e4fe8001e80fb0037
:10c0b000218c200091009000810f5000f4ff390086
:10c0c0000080fa00000006000e00fa0020479800e9
:10c0d0000040eb00004f7800a9c8bf00e14f5000be
:10c0e00003003200adc8bf00e14f500002003a002b
:10c0f00010c0b300004f78002e409000fd4f50005c
:10c1000050003600ae40900070c2b30080cf5000a7
:10c110004c003e001e04e0003e0032002e40900025
:10c120000080fb006101b90020fe2f00f1ff2f000d
:10c1300002014000838148003207980043079800bd
:10c1400090002000010020003e019000ce019000f0
:10c15000800f5100818f59002a003e003e00900060
:10c16000ce00900000600100090037000b0037008e
:10c170000d0037000f0037001100370013003700a3
:10c180001500370017003700190037001b00370073
:10c1900010c2b300104798001a00370000c4b30063
:10c1a000104798001700370030c2b30010479800be
:10c1b0001400370040c2b300104798001100370048
:10c1c00050c2b300104798000e003700e0c5b3001e
:10c1d000104798000b00370060c2b300104798006a
:10c1e00008003700a0c2b3001047980005003700d0
:10c1f00080c2b300104798000200370090c2b3001d
:10c20000104798001e4090000080fb002007980017
:10c21000cd003700ae40900070c2b30080cf500018
:10c2200003003a000103200021079800c6003700f0
:10c230002e409000734040000080fb0020079800d3
:10c24000c1003700ae40900080c5b30080cf5000e1
:10c250000d003600ae40900010c6b30080cf5000f5
:10c2600009003e0023c9bf00e14f500006003a001c
:10c27000ae40900080cdb30000c040000080fb00c5
:10c2800020079800b0003700ae40900020c6b300f1
:10c2900080cf500006003a0023c9bf00e14f500094
:10c2a00003003a000203200022079800a60037008e
:10c2b0002e409000e34f50001f0036002e409000ab
:10c2c000fd4f50001c003e0022c9bf00e14f50004e
:10c2d00006003a00a9c8bf000004e00003003a00cd
:10c2e000adc8bf000004e0000900320022c9bf0051
:10c2f0000004e0000b003a00a9c8bf00e14f500065
:10c3000003003200adc8bf00e14f500005003a0005
:10c310002e409000d043b0000080fb002007980022
:10c32000890037002e409000d045b0000080fb000f
:10c330002007980084003700ae409000c0c2b300d0
:10c3400080cf50007e003600ae40900080c3b30026
:10c3500080cf50007a003e002e4090000080fb000d
:10c360006101b90030fd2f00f1ff2f0002014000f4
:10c37000838148005207980063079800b0002000ae
:10c38000010020005e019000ee019000800f51003e
:10c39000818f590066003e005e009000ee00900024
:10c3a000006001000b003700120037001900370051
:10c3b00020003700270037005d0037002d003700d0
:10c3c000340037003b003700420037004900370097
:10c3d000500037001e04e00003003a00d0c2b30052
:10c3e0001047980052003700f0c5b300104798007e
:10c3f0004f0037001e04e00003003a00d0c3b30032
:10c40000104798004a003700b0c2b30010479800a8
:10c41000470037001e04e00003003a00b0c5b30037
:10c420001047980042003700b0c7b300104798008b
:10c430003f0037001e04e00003003a00d0c5b300ff
:10c44000104798003a003700d0c7b3001047980053
:10c45000370037001e04e00003003a00c0c5b300f7
:10c460001047980032003700c0c7b300104798004b
:10c470002f0037001e04e00003003a00b0c3b300f1
:10c48000104798002a003700a0c3b3001047980057
:10c49000270037001e04e00003003a0070c2b3001a
:10c4a000104798002200370020c2b30010479800c0
:10c4b0001f0037001e04e00003003a0000c6b3006e
:10c4c000104798001a003700e0c7b30010479800e3
:10c4d000170037001e04e00003003a00c0c2b3009a
:10c4e0001047980012003700c0c3b30010479800ef
:10c4f0000f0037001e04e00003003a00e0c2b30062
:10c50000104798000a003700e0c3b30010479800b6
:10c51000070037001e04e00003003a00f0c2b30039
:10c520001047980002003700f0c3b300104798008e
:10c530001e4090000080fb0020079800020037009a
:10c540008000eb00210798002e0090000080fa0088
:10c55000000006000600fa002047980031479800c6
:10c56000d0c8bf008080fb00000320000080600076
:10c570004480de0010479800d0c8bf006f4f6000b5
:10c580003e409000fd4f500004003600be40900039
:10c5900070c2b30080cf5000190036003e409000ba
:10c5a000e34f5000030036003e409000fd4f500026
:10c5b00013003600be409000c0c2b30080cf5000d0
:10c5c00004003600be40900080c3b30080cf50000e
:10c5d0000b003600be40900080c5b30080cf5000f5
:10c5e0000d003600be40900020c6b30080cf500042
:10c5f00009003e0023c9bf00e14f500006003a0089
:10c600002e40900010050700d0c8bf000040e80091
:10c61000d0e8b70088003700be40900090c2b30059
:10c6200080cf500005003a00f7040700d604070049
:10c630000040eb00d0e8b7007f003700be4090001c
:10c64000c0c2b30080cf500006003a0000c2b30061
:10c65000fd040700d0c8bf000040e800d0e8b700e4
:10c6600075003700be409000a0c2b30080cf5000dc
:10c670000b003a00d0c8bf000004e0006e0032009a
:10c680000605070000c2b300ef040700030507001a
:10c69000d0c8bf000040e900d0e8b700660037000e
:10c6a000be409000e0c4b30080cf500004003600cc
:10c6b000be40900020c5b30080cf5000130036006c
:10c6c000be409000c0c5b30080cf50000c003200c7
:10c6d000be409000e0c5b30080cf5000080032009b
:10c6e000be409000a0c5b30080cf500004003200cf
:10c6f000be40900000c6b30080cf50004e003a000c
:10c7000023c9bf000004e0004b003a003e40900007
:10c710000080fb002007980020052000ae0090005c
:10c72000808f50003100320020052000ae009000c4
:10c73000808f50000d003c0000052000ae009000ee
:10c74000808f50002400320000052000ae009000d1
:10c75000808f50002f003c00f0042000ae009000bd
:10c76000808f50001700320033003700c0052000d2
:10c77000ae009000808f500017003200c0052000ee
:10c78000ae009000808f500005003c00a005200006
:10c79000ae009000808f50001e003200260037004f
:10c7a000e0052000ae009000808f500005003200b0
:10c7b00000062000ae009000808f50000b00320079
:10c7c0001d003700c0040700d0c8bf000040e800cb
:10c7d000d0e8b70018003700b0040700d0c8bf0089
:10c7e0000040e900d0e8b700130037001e40900079
:10c7f000e14f500010003a00be040700d0c8bf004f
:10c8000070405000d0e8b7000040eb00104798009f
:10c81000090037001e4090000004e00006003a00c6
:10c82000cf040700d0c8bf0070404000d0e8b70078
:10c8300010c0b30010479800d0c8bf008080fb0034
:10c8400000032000008060004480de001047980054
:10c85000d0c8bf006f4f60001e409000e14f5000f5
:10c8600006003a001e04e00004003a0056040700e7
:10c8700000c1b300d0e8b700090037001e409000a7
:10c88000e24f500006003a001e04e00004003a00a7
:10c890005d0407003c0407000040eb00d0e8b7004f
:10c8a000018d20009140780000c2b30080cf50007d
:10c8b0000400360054040700330407000040eb0076
:10c8c000d0e8b7000080fa00000006000600fa0079
:10c8d00010079800414798000040eb00004f780097
:10c8e0004e409000e14f500010003a00260407002f
:10c8f000070037001e009000104078005204070027
:10c900001e4fe8001e0090000000e800100798008d
:10c910001e009000104078000004e000f5ff3a008f
:10c92000f0c0b3009e4f1000f2ff36004e40900062
:10c93000e24f500010003a002304070007003700c0
:10c940001e009000104078003f0407001e4fe800d2
:10c950001e0090000000e800100798001e009000e4
:10c96000104078000004e000f5ff3a00f0c0b3008a
:10c970009e4f1000f2ff36000080fa000000060013
:10c980001400fa000040eb00305798000000eb0064
:10c99000300798000000eb00200798000000eb0033
:10c9a00010079800208220007007980080872000e0
:10c9b000000f98000000eb00000f78007e00900050
:10c9c000e0689000315798000040eb002057980035
:10c9d000be0037000e089000300190002e509000ed
:10c9e0008080fb00e00220000088b90000004100c8
:10c9f000600798006e009000100078000000e000d2
:10ca00003f003a006e00900020119000b01190009d
:10ca10002000200001002000800f5100818f59006c
:10ca200037003a006e00900010009000e70f5000b1
:10ca300033003a006e00900080689000114f98001b
:10ca40000e089000600190001e4890000080fb00de
:10ca50006a00b90000004100500798005e00900095
:10ca6000b0009000000e2000808f500094003a002b
:10ca70005e009000c0009000700e2000808f50007b
:10ca80008f003a006e00900060089000004f980000
:10ca90000e089000c00090000e4890000080fb003f
:10caa0004300dd000080400010009000670040005f
:10cab0004300de00a04488006e00900060589000a3
:10cac0000080fb00b04488006e0090002060900061
:10cad00098e8b7006e0090007058900099e8b70091
:10cae0006e009000006090009ae8b7006f010700a8
:10caf0009ce8b70010002000200798007000370065
:10cb00006e009000100078000000e0003c003a0049
:10cb10006e009000b010900020109000e00f5000c8
:10cb2000e08f580036003a006e0090001000900030
:10cb3000e70f500032003a006e00900080689000cd
:10cb4000114f98000e089000600190001e48900060
:10cb50000080fb006a00b900000041005007980007
:10cb60005e009000300090000000e00054003a00a9
:10cb70005e009000c0009000f00f2000808f5000f9
:10cb80004f003e006e00900060089000004f98003b
:10cb90000e089000c00090000e4890000080fb003e
:10cba0004300dd000080400010009000670040005e
:10cbb0004300de00f04488006e0090006058900052
:10cbc0000080fb00004588006e009000206090000f
:10cbd000a2e8b7006e00900070589000a3e8b7007c
:10cbe0006e00900000609000a4e8b7002f010700dd
:10cbf000a6e8b700100020001007980030003700aa
:10cc00006e00900010007800e10f50002c003a00f8
:10cc10006e00900010009000e80f500028003a00cd
:10cc20006e00900080689000114f98000e089000f0
:10cc3000600190001e4890000080fb006a00b9006f
:10cc400000004100500798006e00900060089000be
:10cc5000004f98000e089000c00090000e48900011
:10cc60000080fb004300dd000080400020009000b9
:10cc7000670040004300de00504488006e009000d2
:10cc8000605890000080fb00604488006e009000b7
:10cc9000206090008ee8b7006e0090007058900001
:10cca0008fe8b7006e0090000060900090e8b70039
:10ccb000fe00070092e8b70010002000300798003f
:10ccc0002e5090000040e80020579800ae50900091
:10ccd0003e50900080cf50003eff39007e00900013
:10cce00070689000e14f500020003a00218c200035
:10ccf0000000eb00800878000e089000c000900053
:10cd00000e4890000080fb004300dd0000804000e2
:10cd10001000900067004000c300de00208c20005f
:10cd200011009800208c20001000900003d707000d
:10cd300080007800208c2000210098007e00900068
:10cd400090007800208c2000310098001e00900098
:10cd5000e10f500005003a002e009000e10f500056
:10cd600002003a0010002000000f78001e0078003a
:10cd70000080fa00000006000200fa00810a20008c
:10cd80009140780080cfb30000c060000004a00094
:10cd9000a8e0b7008500a9000000eb00500888005b
:10cda000208c200030009000a2002000110009001b
:10cdb0000280d8008000780000e224000088b900da
:10cdc000000f780000e224007008880000012a00ab
:10cdd000900888009500a8000080fa000000060076
:10cde000801f78003400f80000c0b300a001880064
:10cdf0000000fa0085c0bf00614060000004e00050
:10ce0000060032008500a900d0488000e20f5000e3
:10ce100002003a0030002000d04888000080fa006c
:10ce20003400f9004f007800004006000800fa00c6
:10ce3000004f78001207980023079800407a2900d5
:10ce40008f0307002ac9bf000004e00005003a0074
:10ce50001e4078002ae9b700100020003007980033
:10ce6000020037000000eb00300798003e00900001
:10ce70000080fa00000006000e00fa00004f780063
:10ce8000110798002207980034079800450798007a
:10ce90002ac9bf009e4f50003c003a001e0090007f
:10cea00060079800d0122000ee009000808f5000a4
:10ceb0001f003200d0122000ee009000808f500042
:10cec0000b003e006e009000e80f50002100320081
:10ced000c0122000ee009000808f50001100320040
:10cee0006e009000e70f5000200032002400370051
:10cef000f0122000ee009000808f500020003900da
:10cf000010132000ee009000808f500005003600c6
:10cf100020132000ee009000808f5000100032009f
:10cf20001700370010002000500798001900370044
:10cf300093fe07000000e000030032001100200013
:10cf400051079800130037000000eb0050079800cd
:10cf50001000370011002000510798000d00370025
:10cf600010002000500798000a0037000040eb0036
:10cf70002ae9b7001100200051079800050037008a
:10cf80000000eb0050079800020037008000eb0023
:10cf9000510798005e0090000080fa000000060033
:10cfa0000200fa00b0d9070084ea07002ac9bf00ce
:10cfb000c9e907008040780030c5b30080cf500039
:10cfc00006003a002ac9bf000004e0000300320056
:10cfd00010002000000f7800020037000000eb0076
:10cfe000000f78001e0078000080fa0000000600a4
:10cff0000600fa00000f7800214798003247980099
:10d00000230798003e4090000080fb00a69220007d
:10d0100016437800ae029000000278009e0178006e
:10d020002e41900011c0b3000640780021ef0700a8
:10d030000080fb000080fa00000006000600fa00f5
:10d04000000f780021479800324798002307980086
:10d050003e4090000080fb00a6922000164378001e
:10d06000ae029000000278009e0178002e419000f0
:10d070008040eb00064078000eef07000080fb00c8
:10d080000080fa00000006000400fa00000f78009b
:10d09000110798002ac9bf001e0190009e00780069
:10d0a000a2ef07000080fa00000006000000fa006e
:10d0b00057c8bf000080fb000080fa000000060097
:10d0c0001e00fa0050079800610798007207980048
:10d0d000030f9800140f9800250f98000040eb00f4
:10d0e000505f98000e0890000000e00002003a0037
:10d0f00011c0b300515f98000041eb00425f9800ff
:10d100001e0890000000e00002003a0010c0b300ca
:10d11000405f9800de5890004e59900002c07000a9
:10d120000080fb00500f98000000eb00400f9800bb
:10d130002e0890000000e00002003a0011002000dc
:10d14000410f98005e099000ce0890000100710028
:10d150000000e000030032000001eb00320f9800f5
:10d160005b0037000000eb002007980051003700fb
:10d17000f2438000ae009000e00220000088b90079
:10d18000000f41001e007800900078007e009000a3
:10d19000808f500044003a0068004700e6004700d6
:10d1a00000027800810178006e019000de0090009e
:10d1b0001e007800e9f807000000e0003a003200a5
:10d1c0001e007800e00890001107980001448000dc
:10d1d0001e0090004300dd00008040001000780039
:10d1e000804078000e089000014878001e0078000a
:10d1f000a06090003e00900080c040002e0890008b
:10d20000014878007e0090000000e0000b003a002a
:10d21000014480001e0090004300dd0000804000bb
:10d2200010009000670040004300de00804078005e
:10d230001e08900001487800180037007e0090001a
:10d24000e10f50000b003a00014480001e009000e6
:10d250004300dd0000804000200090006700400097
:10d260004300de00804078001e08900001487800ee
:10d270000a003700014480001e0090004300dd00da
:10d280000080400030009000670040004300de0056
:10d29000804078001e0890000148780012002000ad
:10d2a000320f98000a0037002e0090000000e800be
:10d2b0002007980050c8bf008080fb002e0090001f
:10d2c000808f5000aaff3e000000eb00300f980056
:10d2d0003e0890000080fa00000006002400fa00da
:10d2e000500798006107980072079800030f980094
:10d2f000140f9800250f9800360f98000040eb009f
:10d30000306798000e0890000000e00002003a002c
:10d3100011c0b300316798000041eb00226798000c
:10d320001e0890000000e00002003a0010c0b300a8
:10d3300020679800be6090002e61900002c07000cf
:10d340000080fb00001798000000eb00700f9800b1
:10d350002e0890000000e00002003a0011002000ba
:10d36000710f98000e1190007e089000000171006e
:10d37000620f98008000eb00510f98003e0890006b
:10d380000000e00002003a0012002000520f980056
:10d39000ee0890005e099000028070000000e0003e
:10d3a000030032000000eb00400f980070003700cf
:10d3b0000040eb002047980066003700f2438000f1
:10d3c0002e4090008080fb00e00220000088b90021
:10d3d000000f41001e007800900078007e00900051
:10d3e000808f500058003a001e007800b010900066
:10d3f000201090008100d1000080d3006100600007
:10d400000004e000500032001e00780070589000c8
:10d41000e14f50004c00320068004700e600470032
:10d4200000027800810178006e019000de0090001b
:10d430001e00780049f807000000e00042003200ba
:10d440001e007800e0089000210798000144800049
:10d450002e0090004300dd000080400010007800a6
:10d46000804078000e089000014878001e00780087
:10d47000f05890003e089000014878001e007800a7
:10d48000206190001e007800705890008080fb00a2
:10d490003e0090000088b900804041002e089000b6
:10d4a000014878007e0090000000e0000b003a0088
:10d4b000014480002e0090004300dd000080400009
:10d4c00010009000670040004300de0080407800bc
:10d4d0001e08900001487800180037007e00900078
:10d4e000e10f50000b003a00014480002e00900034
:10d4f0004300dd00008040002000900067004000f5
:10d500004300de00804078001e089000014878004b
:10d510000a003700014480002e0090004300dd0027
:10d520000080400030009000670040004300de00b3
:10d53000804078001e08900001487800120020000a
:10d54000420f98000a0037002e4090000040e8008b
:10d550002047980001852000914078002e409000df
:10d5600080cf500095ff3e000000eb00400f980078
:10d570004e0890000080fa00000006001e00fa002d
:10d58000100f9800210f9800320f9800430f980059
:10d590001e0890000000e00003003a000000eb00cd
:10d5a000600f9800ae0037004e0890001000900009
:10d5b0000000e0000a0032004e0890009000900049
:10d5c0001e089000104078000080fb00808f500003
:10d5d000030032000000eb00600f9800a00037004d
:10d5e0004e089000900078002e089000808f500028
:10d5f000030032000000eb00600f98009800370035
:10d600004e089000404090000081fb004e089000c2
:10d61000504090008080fb004e08900060409000d9
:10d620000080fb000088b900000041000000e90014
:10d6300082002000110009000200d80010079800a5
:10d640009e0090002e089000808f5000030036004e
:10d650000000eb00600f9800810037004e0890003a
:10d66000404090000080fb00400798000000eb0065
:10d67000000f7800730037004e0090004300de007a
:10d68000300798004e009000670060002007980067
:10d690004e089000504090008080fb004e009000ab
:10d6a000008040000000e9004300de001007980001
:10d6b0000000eb00000f98000e0890004800dd000d
:10d6c000000f98009e0090001e089000008040000f
:10d6d000104078008080fb000e0890000100700070
:10d6e000000f98000040eb00205f98009e00900023
:10d6f0003e009000808f50000200360010c0b30042
:10d70000205f98001e0090000000e90010079800bc
:10d710002e5890000004e000e7ff3a002e00900031
:10d720000000e000040032002e0090008e089000ff
:10d730000008de00000f98004e0890005040900056
:10d74000ef4f500031003e004e08900050409000d6
:10d750008080fb00100020000100dd0060079800c1
:10d760006e0090000000e900600798008e089000ad
:10d770006e00900000806000000f98004e0890003e
:10d78000704090000004e0002000320010002000f3
:10d79000700798004e08900050409000e14f5000f4
:10d7a000070036004e089000504090000080fb00bb
:10d7b0008000e9007e0090000100dd007007980005
:10d7c0007e009000000040000000e9005007980033
:10d7d0008e0890007e009000008060000000e00055
:10d7e00005003a000e089000de0090000100600085
:10d7f000000f9800050037005e0090008080ea006e
:10d800000e08900001007000000f98000e089000b4
:10d81000804078003e089000014878003e08900063
:10d820000000e800300f98004e0890005040900033
:10d830008080fb004e0090000100400040079800ef
:10d840001e0fe8004e089000604090000080fb0032
:10d850009e0f500088ff3e0010002000600f9800cf
:10d860006e0890000080fa00000006000000fa0038
:10d8700000e224004049880040498000d3000700ae
:10d880004006200040498800800320004030880086
:10d8900040498000cd00070000e224004049880094
:10d8a00040498000c9000700400620004049880028
:10d8b000c00020004030880040498000c3000700bd
:10d8c00000e224004049880040498000bf00070072
:10d8d00080bb2000404988001000200040308800b4
:10d8e00040498000b900070000e224004049880058
:10d8f00040498000b500070080bb200040498800f7
:10d90000f00020004030880040498000af00070050
:10d9100000e224004049880040498000ab00070035
:10d9200080bb200040498800600020004030880013
:10d9300040498000a50007003300070002000700ef
:10d940000080fa00000006000000fa0080bb200002
:10d95000404988000000eb002030880020002000b3
:10d960004030880003003700404980000000e90093
:10d9700040498800404980000000e000faff3a007a
:10d980000080fa00000006000000fa0080bb2000c2
:10d99000404988000000eb0020308800000820008b
:10d9a0004030880003003700404980000000e90053
:10d9b00040498800404980000000e000faff3a003a
:10d9c0000080fa00000006000000fa0080bb200082
:10d9d000404988000000eb0020308800000c200047
:10d9e0004030880003003700404980000000e90013
:10d9f00040498800404980000000e000faff3a00fa
:10da00000080fa00000006000000fa0080bb200041
:10da1000404988000000eb00203088001000200002
:10da20004030880003003700404980000000e900d2
:10da300040498800404980000000e000faff3a00b9
:10da40000080fa00000006000200fa00004f780093
:10da50004006200040498800100020002030880047
:10da60001e00fb0040308800030037004049800062
:10da70000000e90040498800404980000000e000c3
:10da8000faff3a0000000000000000000000000063
:10da9000000000000080fa00000006000000fa000c
:10daa00040062000404988000000eb00203088003c
:10dab00000012000403088004049800043000700fa
:10dac0000080fa00000006000000fa004006200076
:10dad000404988000000eb00203088004001200011
:10dae0004030880040498000380007000080fa007c
:10daf000000006000200fa004006200040498800ad
:10db00000000eb0020308800c0002000403088007a
:10db1000404980002d0007000040eb00004f7800d6
:10db200002003700ddff07001e4fe800f0c0b30021
:10db30009e4f1000fbff3600400620004049880041
:10db40000000eb0020308800f0002000403088000a
:10db5000404980001d0007000080fa000000060018
:10db60000200fa0040062000404988000000eb0057
:10db700020308800c00020004030880040498000ec
:10db8000120007000040eb00004f78000200370051
:10db9000cdff07001e4fe800f0c0b3009e4f1000fd
:10dba000fbff360040062000404988000000eb00e3
:10dbb00020308800f000200040308800404980007c
:10dbc000020007000080fa00000006000200fa00d0
:10dbd000000f7800010037001e0fe9001e00e00072
:10dbe000fdff3a000080fa00000006000200fa0083
:10dbf00087c0bf000044b2000004e000fcff320018
:10dc0000b0118000004f780087c0a9001e00fb0003
:10dc10000080fa00000006000000fa004004200026
:10dc2000c01188000000eb00801188003062a8005d
:10dc30000000eb009011880031e2a8003342a800f8
:10dc400087c0a9000080fa00000006000200fa0068
:10dc500087c0bf000044b2000004e00003003200af
:10dc600010002000000f7800020037000000eb00d9
:10dc7000000f78001e0078000080fa000000060007
:10dc80000600fa0010079800020037001e407800d6
:10dc9000120007001e00900010407800004f78002e
:10dca0001e407800404798004e4090000004e0007d
:10dcb0000200320010c0b300404798004e40900070
:10dcc0009e0090008100e800110798000004e00029
:10dcd000eeff3a000080fa00000006000200fa00a1
:10dce000004f78001e00fb00a0118800000000001b
:10dcf00033c2bf00614060000004e000fcff32005e
:10dd00000080fa00000006000400fa002047980096
:10dd10002e409000004f780030c6b3009e4f100098
:10dd2000060036001e80fb0042062000110009009c
:10dd30000280d8000043b000e8ff07009e41780051
:10dd40001e80fb0042062000110009000280d8005e
:10dd50008080fb00400620000088b90000c0510010
:10dd6000004f780090c0b3009e4f100006003600b0
:10dd70001e80fb00a2002000110009000280d800d4
:10dd80000043b000d5ff07009e4178001e80fb00d5
:10dd9000a2002000110009000280d8000080fb00d2
:10dda0006a00b90000c05100004f78001e407800a2
:10ddb0000043b000c9ff07000080fa000000060021
:10ddc0000400fa00100798001e009000000f780071
:10ddd0001e0090004480de006f0060001007980075
:10dde0009e009000c07b290061407800bbff0700c7
:10ddf0009e0078006f806000100798009e009000e1
:10de0000c07b290061407800b4ff07000080fa0061
:04de10000000060008
:020000040000fa
:10de1400d2080000280000000200000016673c0041
:10de2400670000000000ce00482648000000000003
:10de340000ce480026480000000000000301010055
:10de440000000000020003000000000000000200c7
:10de5400000000001a0900000a000000020000008f
:10de640000000000000000000000000000000000ae
:10de74008a08000048000000000000002809000093
:10de8400020000000000000024090000040000005b
:10de9400020000000000000000000000fa0800007a
:10dea40014000000000000002a0900000200000025
:10deb40002000000000000002208000068000000ca
:10dec400020000000000000000000000000000004c
:10ded400000000000000000000000000000000003e
:10dee400000000000000000000000000000000002e
:10def400000000000000000000000000000000001e
:10df0400000000000000000000000000000000000d
:10df140000000000000000000000000000000000fd
:10df240000000000000000000000000000000000ed
:10df340000000000000000000000000000000000dd
:10df440000000000000000000000000000000000cd
:10df54000e0900000c000000020000000000000098
:10df6400000000000000000000000000000a0000a3
:10df74001000000000000000000800002200000063
:10df8400000000002e09000006000000020000004e
:10df940000020000000000002c0900000200000044
:08dfa400000000000000000075
:020000040000fa
:04dfac000000fe0073
:00000001FF
